:1000000000000120910400003B0600003D060000B6
:100010003F060000410600004306000039060000CC
:1000200039060000390600003906000045060000C8
:100030004706000039060000490600004B06000094
:100040004D0600004F060000510600005306000058
:100050005506000057060000590600005B06000028
:100060005D0600005F0600006106000063060000F8
:100070006506000067060000690600006B060000C8
:100080006D0600006F060000710600007306000098
:100090007506000077060000790600007B06000068
:1000A0007D0600007F060000810600008306000038
:1000B0008506000087060000890600008B06000008
:1000C000390600008D060000390600008F0600008A
:1000D00039060000390600003906000091060000CC
:1000E000930600009506000039060000390600005E
:1000F0009706000039060000990600009B060000E4
:100100009D0600009F060000A1060000A306000057
:10011000A506000039060000390600003906000077
:1001200039060000A7060000A9060000AB06000083
:10013000AD060000AF060000B1060000B3060000E7
:1001400039060000390600003906000039060000B3
:10015000B506000039060000390600003906000027
:100160003906000039060000390600003906000093
:100170003906000039060000B7060000B906000085
:10018000BB060000BD060000BF060000C10600005F
:10019000C3060000C5060000C7060000C90600002F
:1001A000CB060000CD060000CF060000D1060000FF
:1001B000D3060000D5060000D7060000D9060000CF
:1001C000DB060000DD060000DF060000E10600009F
:1001D000E3060000E5060000E7060000E90600006F
:1001E000EB060000ED060000EF060000F10600003F
:1001F000F3060000F5060000F7060000F90600000F
:10020000FB060000FD060000FF06000001070000DD
:1002100003070000050700000707000009070000AA
:100220000B0700000D0700000F070000110700007A
:10023000130700001507000017070000190700004A
:100240001B0700001D0700001F070000210700001A
:1002500023070000250700002707000039060000DB
:100260003906000039060000390600003906000092
:100270003906000039060000390600003906000082
:100280003906000039060000390600003906000072
:100290003906000039060000390600003906000062
:1002A0003906000039060000390600003906000052
:1002B000290700002B0700002D0700002F07000072
:1002C0003107000033070000350700003707000042
:1002D000390700003B0700003D0700003F07000012
:1002E00041070000430700004507000047070000E2
:1002F000490700004B0700004D0700004F070000B2
:1003000039060000390600005107000053070000BD
:100310005507000057070000590700003906000084
:10032000390600005B0700005D0700005F07000062
:0C03300061070000630700006507000083
:100400000004FF1F600B0000600B000001000000F3
:100410000004FF1F640B0000640B000001000000DB
:1004200014490C684FF001031C401349134A521A37
:10043000013A06DD4FF05A304FF05A3309C1083AFD
:10044000FCDA0F490F4A521A013A06DD4FF05A30D2
:100450004FF05A3309C1083AFCDA0B490B4A521AD9
:10046000013A06DD4FF05A304FF05A3309C1083ACD
:10047000FCDA704700F007400000FF1F0004FF1F78
:1004800000FC0020000001200004FF1F00FC0020F1
:1004900072B64FF000014FF000024FF000034FF032
:1004A00000044FF000054FF000064FF00007B8467B
:1004B000B946BA46BB46BC46FFF7B2FF064885467A
:1004C00006488047064880470648804706488047D8
:1004D00062B600F00BF8FEE700000120F104000016
:1004E000F905000069070000F505000000BFFDE701
:1004F000F0B583B03A4B1D680023009302230093AC
:10050000009B002B3ED005F00105364C4FF0000C4F
:1005100031E055B35668116893689B1B03F00302E2
:100520008DF807209DF807209B1A5FEA930E09D0EB
:10053000331F0A1F03EB8E0753F8040F42F8040F12
:10054000BB42F9D14FEA8E039DF807206AB1F21839
:10055000581E0144164612F8013B01F8013F9DF870
:100560000730DBB2901B8342F5D80CF1010C009BE5
:100570001034634506D92246237B022BC9D0002BB9
:10058000F3D0C7E701230093009B33B3164C174AFF
:10059000121B02F003038DF807309DF80730D21AC2
:1005A000920807D004EB82002346002143F8041B85
:1005B0008342FBD192009DF807306BB10C48104488
:1005C0000025034600F8015F9DF80710C9B2023309
:1005D0001B1B9B1A9942F4D8009B03B0F0BD00BFCF
:1005E00000F00740000400000004FF1F0004FF1F8C
:1005F000FF03FF1F7047000008B500F0D9F80B4A51
:100600000B4B9B1A032B0AD94FEA930C0949002381
:1006100052F8040B41F8040B01339C45F8D8054A05
:100620004FF0E023C3F8082D08BD00BF0000000014
:100630003C0300000000FF1FFEE7FEE7FEE7FEE7C9
:10064000FEE7FEE7FEE7FEE7FEE7FEE7FEE7FEE782
:10065000FEE7FEE7FEE7FEE7FEE7FEE7FEE7FEE772
:10066000FEE7FEE7FEE7FEE7FEE7FEE7FEE7FEE762
:10067000FEE7FEE7FEE7FEE7FEE7FEE7FEE7FEE752
:10068000FEE7FEE7FEE7FEE7FEE7FEE7FEE7FEE742
:10069000FEE7FEE7FEE7FEE7FEE7FEE7FEE7FEE732
:1006A000FEE7FEE7FEE7FEE7FEE7FEE7FEE7FEE722
:1006B000FEE7FEE7FEE7FEE7FEE7FEE7FEE7FEE712
:1006C000FEE7FEE7FEE7FEE7FEE7FEE7FEE7FEE702
:1006D000FEE7FEE7FEE7FEE7FEE7FEE7FEE7FEE7F2
:1006E000FEE7FEE7FEE7FEE7FEE7FEE7FEE7FEE7E2
:1006F000FEE7FEE7FEE7FEE7FEE7FEE7FEE7FEE7D2
:10070000FEE7FEE7FEE7FEE7FEE7FEE7FEE7FEE7C1
:10071000FEE7FEE7FEE7FEE7FEE7FEE7FEE7FEE7B1
:10072000FEE7FEE7FEE7FEE7FEE7FEE7FEE7FEE7A1
:10073000FEE7FEE7FEE7FEE7FEE7FEE7FEE7FEE791
:10074000FEE7FEE7FEE7FEE7FEE7FEE7FEE7FEE781
:10075000FEE7FEE7FEE7FEE7FEE7FEE7FEE7FEE771
:10076000FEE7FEE7FEE7000008B50D4AD2F8883044
:1007700043F47003C2F888300A4A136843F08023B8
:100780001360094B4BF231621A604CF278221A6006
:100790005A6822F001025A60044800F00BF808BDC4
:1007A00000ED00E00000014000A00640B408000099
:1007B0000020704770B53D4BD3F89040C4F3072438
:1007C000BFF35F8F5A6A22F480325A62D3F89420C2
:1007D00022F00102C3F89420BFF34F8FBFF36F8F55
:1007E00054B10023314A1D46C2F89830C2F8A050D7
:1007F0000133D9B28C42F7D8C37823B300212C4CF3
:100800004FF0FF0C04E00131C278CBB29A421AD902
:10081000CBB2426802EB430612F81330072BF2D832
:1008200003F0030E4FEACE0E03F0FC0323441D6BCE
:10083000727802FA0EF26A400CFA0EFE02EA0E021A
:100840006A401A63DFE7037AB3B100221749D3B2D3
:1008500003EB4303C56805EB830415F82360656863
:10086000A368C1F89860C1F89C50C1F8A03001326B
:10087000047AD3B29C42EAD80378012B14BF002338
:1008800004234278012A08BF43F00203BFF35F8FBD
:1008900043F00103054AC2F89430536A43F48033AD
:1008A0005362BFF34F8FBFF36F8F70BD00ED00E059
:1008B00090ED00E0010001021809000007000000AF
:1008C000C40800000000000006000000E1FF0F0067
:1008D0000100000007001000E1FF1300020000000B
:1008E00001000010E10300100300000001000110EE
:1008F000E10301100400000001000310E1030310F4
:10090000050000000200FF1FE1FF002006000000BC
:0C09100001000040E3FF0740004401002C
:040000030000049164
:00000001FF
